:10000000F9C500001FC600001DC600001BC6000089
:1000100019C6000017C6000015C6000013C6000070
:1000200011C600000FC600000C945A150C94C91597
:1000300009C6000007C6000005C6000003C6000090
:1000400001C60000FFC50000FDC50000FBC50000A3
:10005000F9C50000F7C50000F5C500000C941015A7
:10006000F1C50000EFC50000EDC50000EBC50000C4
:10007000E9C50000E7C50000E5C50000E3C50000D4
:10008000E1C50000DFC50000DDC50000DBC50000E4
:10009000D9C50000D7C50000D5C50000D3C50000F4
:1000A000D1C50000CFC50000CDC50000D5F08D142E
:1000B000A1C881CFD9F1AF20005072657373204180
:1000C00020666F72206D656E750053746172733AAD
:1000D00020004B696C6C733A200044657074683A78
:1000E000200047616D65204F766572005374616929
:1000F0006E6C65737300436C61796D6F7265004B54
:100100006174616E6100537465656C2053776F7222
:10011000640049726F6E2053776F726400496E639A
:100120006F6E63656C204368657374005374616916
:100130006E6C6573732043686573740053746565F2
:100140006C2043686573740049726F6E2043686564
:10015000737400496E636F6E656C2050616E7473CA
:1001600000537461696E6C6573732050616E7473B3
:1001700000537465656C2050616E74730049726F32
:100180006E2050616E747300496E636F6E656C20F3
:1001900048656C6D00537461696E6C6573732048BB
:1001A000656C6D00537465656C2048656C6D004925
:1001B000726F6E2048656C6D00496E636F6E656C82
:1001C00020426F6F747300537461696E6C65737352
:1001D00020426F6F747300537465656C20426F6FBB
:1001E00074730049726F6E20426F6F747300476FB3
:1001F0006C64204170706C65004368726F6D6500BF
:10020000496E636F6E656C00537465656C0043687E
:10021000726F6D6520496E676F7400476F6C642064
:10022000496E676F74004E69636B656C20496E6739
:100230006F740049726F6E20496E676F7400F0F83A
:100240009C8E8783878E9CF8F00000FEFF030303DB
:100250000303070EFCF80000FEFF0303030303077C
:100260000EFCF80000FFFF00000000000000FFFF90
:100270000000FEFF8383838383C7EE7C380000F891
:10028000FC0E07030303070EFCF800003F7FE0C0ED
:100290008080C0E07F3FFFFF01010101010101FFFC
:1002A000FF0000FFFF0C0C0C0C1C3E77E3C10000AC
:1002B0007FFFC0C0C0C0C0E0703F1F00001F3F7084
:1002C000E0C0C0C0E0703F1F00007FFFC1C1C1C1DE
:1002D000C1E3773E1C00001F3F70E0C0C0C0E0706B
:1002E0003F1F000000000001FFFF010000000000B0
:1002F0000000003E5B4F5B3E3E6B4F6B3E1C3E7C06
:100300003E1C183C7E3C181C577D571C1C5E7F5EB3
:100310001C00183C1800FFE7C3E7FF001824180072
:10032000FFE7DBE7FF30483A060E26297929264009
:100330007F050507407F05253F5A3CE73C5A7F3E35
:100340001C1C08081C1C3E7F14227F22145F5F00C7
:100350005F5F06097F017F006689956A6060606063
:100360006094A2FFA29408047E040810207E20104E
:1003700008082A1C08081C2A08081E101010100C57
:100380001E0C1E0C30383E3830060E3E0E060000A5
:1003900000000000005F00000007000700147F1449
:1003A0007F14242A7F2A12231308646236495620B8
:1003B000500008070300001C2241000041221C00DD
:1003C0002A1C7F1C2A08083E08080080703000089C
:1003D00008080808000060600020100804023E5170
:1003E00049453E00427F4000724949494621414902
:1003F0004D331814127F1027454545393C4A494969
:100400003141211109073649494936464949291ED2
:1004100000001400000040340000000814224114C1
:1004200014141414004122140802015909063E4113
:100430005D594E7C1211127C7F494949363E41413B
:1004400041227F4141413E7F494949417F09090994
:10045000013E414151737F0808087F00417F410000
:100460002040413F017F081422417F404040407FAF
:10047000021C027F7F0408107F3E4141413E7F09FC
:100480000909063E4151215E7F091929462649493D
:10049000493203017F01033F4040403F1F2040207D
:1004A0001F3F4038403F631408146303047804037B
:1004B0006159494D43007F41414102040810200029
:1004C0004141417F0402010204404040404000039A
:1004D00007080020545478407F2844443838444466
:1004E0004428384444287F385454541800087E095E
:1004F0000218A4A49C787F0804047800447D40007E
:100500002040403D007F1028440000417F40007C97
:10051000047804787C080404783844444438FC188F
:1005200024241818242418FC7C0804040848545473
:10053000542404043F44243C4040207C1C204020A0
:100540001C3C4030403C44281028444C9090907C07
:100550004464544C44000836410000007700000019
:100560004136080002010204023C2623263C1EA15B
:10057000A161123A4040207A3854545559215555BA
:10058000794121545478412155547840205455796B
:10059000400C1E52721239555555593954545459FC
:1005A00039555454580000457C410002457D4200B5
:1005B00001457C40F0292429F0F0282528F07C54BE
:1005C0005545002054547C547C0A097F49324949DE
:1005D00049323248484832324A4848303A4141214B
:1005E0007A3A42402078009DA0A07D3944444439A5
:1005F0003D4040403D3C24FF2424487E4943662B37
:100600002FFC2F2BFF0929F620C0887E09032054D8
:100610005479410000447D413048484A32384040D6
:10062000227A007A0A0A727D0D19317D2629292F36
:1006300028262929292630484D402038080808084E
:1006400008080808382F10C8ACBA2F102834FA0050
:10065000007B000008142A142222142A1408950092
:10066000220095AA005500AAAA55AA55AA00000082
:10067000FF00101010FF00141414FF001010FF00F2
:10068000FF1010F010F0141414FC001414F700FF05
:100690000000FF00FF1414F404FC141417101F10C2
:1006A000101F101F1414141F00101010F000000071
:1006B000001F101010101F10101010F0100000007C
:1006C000FF101010101010101010FF10000000FF8D
:1006D000140000FF00FF00001F10170000FC04F4CE
:1006E00014141710171414F404F40000FF00F71486
:1006F000141414141414F700F7141414171410100D
:100700001F101F141414F4141010F010F000001F28
:10071000101F0000001F14000000FC140000F01067
:10072000F01010FF10FF141414FF141010101F000D
:10073000000000F010FFFFFFFFFFF0F0F0F0F0FF0F
:10074000FFFF0000000000FFFF0F0F0F0F0F3844E6
:100750004438447C2A2A3E147E02020606027E02A7
:100760007E0263554941633844443C04407E201E68
:100770002006027E020299A5E7A5991C2A492A1C97
:100780004C7201724C304A4D4D303048784830BC84
:10079000625A463D3E494949007E0101017E2A2AAE
:1007A0002A2A2A44445F444440514A444040444A2F
:1007B00051400000FF0103E080FF000008086B6B60
:1007C000083612362436060F090F060000181800E6
:1007D00000001010003040FF0101001F01011E0049
:1007E000191D1712003C3C3C3C0000000000080BA7
:1007F00000020202000009040000010202000005DC
:100800002400100105240101010424020605240628
:1008100000010705810310004009040100020A00DD
:1008200000000705020240000007058302400000A7
:100830000403090412010002EF0201404123368043
:1008400000010102030141726475696E6F204C4C16
:100850004300414241313330360042792040426505
:10086000726761736D7300415244554D494E455254
:1008700000536F756E64004C6F6164005374617255
:100880007400674170706C65004170706C65005356
:100890007461696E6C65737300496E636F6E656C2D
:1008A00000537465656C004368726F6D6520496E16
:1008B000676F74004E69636B656C20496E676F7477
:1008C00000476F6C6420496E676F740049726F6EE9
:1008D00020496E676F74004E69636B656C204F72C0
:1008E0006500436F616C004368726F6D65204F72E5
:1008F0006500476F6C64204F72650049726F6E200F
:100900004F726500456D707479005C007C002F00AB
:1009100041200078000209290A212A1211291A19F6
:100920002A2231292C52494129335241293A693E20
:100930004234784A5480536451885B5C51906235EC
:10094000796A5581736551897B5D519182367A8AC6
:1009500057829367528A9B5F5292A337517BAC5761
:10096000615283B46759528BBC5F625293C2327C2E
:10097000CB315284D43151628CDC31525B94E241F0
:1009800029FF4352414654494E4700FF81BDBDBD3A
:10099000BD81FFFF81BDB5ADBD81FFFFA5C993A599
:1009A000C993FFFF819DA7A79D81FFFF83B9E5E55F
:1009B000B983FF102844824122140810386CC661A4
:1009C000321C0810286CAA6B2A1C0810384CE673DD
:1009D0003A1C08C0ACAACA6C505060EEAAAAAAAAD7
:1009E000AAACC03048844221120A04007985858669
:1009F000A55800007985B5CEA55800E09EFE000000
:100A0000FE9EE000786414146478007F4139050587
:100A100039417F007E4C48484C7E006090A0C0C0A9
:100A2000A09060C0A0A0C0C0A0A0C0C0A090606006
:100A300090A0C03649AB2626AB493636C92B1616D0
:100A40002BC936B6492B26262B49B69B35CA101022
:100A5000CA359B1AF58B08088BF51ADA358A08080F
:100A60008A35DA70EA668800000000F069E608005E
:100A700000000070F867480000000070EA66881007
:100A80000D030670E866881010081C70E86788205F
:100A900020C0E070EA668810080C0670E8668810CE
:100AA00010181870E867882060408070EA66880037
:100AB00060600070EA66883030080070EA6688304E
:100AC000000400000000008866EA700000000008D2
:100AD000E669F0000000004867F87006030D108812
:100AE00066EA701C0810108866E870E0C020208854
:100AF00067E870060C08108866EA701818101088ED
:100B000066E870804060208867E870006060008858
:100B100066EA70000830308866EA700004003088A9
:100B200066EA701C3E7C7C3E1CFF81A1958D9981FC
:100B3000FFFF819BBDBD9981FFFF81BD9595BD8163
:100B4000FFFF81BDBDBDBD81FF0000400000000072
:100B500000FEA6CBA6CBA6CBFEFFA593A593A5939F
:100B6000FFFFFFFFFFFFFFFFFFFF81BDBDBDBD8199
:100B7000FFFF83B9E5E5B983FFFF819DA7A79D81AD
:100B8000FFFF81BDB5ADBD81FFAA55AA55AA55AAE3
:100B900055FF81F98989F981FFFFA5C993A5C993FB
:100BA000FFFF9DEB83EBA39DFFFF9DEB83EBA39DDD
:100BB000FFFF81FF81FF81FFFF0000400000000078
:100BC000000000400000000000486F6C64204220DC
:100BD000546F2073617665005072657373204120F5
:100BE000546F20626567696E0044657074683A20CE
:100BF00000002B1811241FBECFEFDAE0DEBFCDBFFF
:100C000011E0A0E0B1E0E6E6F4E502C005900D9247
:100C1000AC34B107D9F727E0ACE4B1E001C01D92D4
:100C2000AC3AB207E1F715E0CAEFD5E004C021976E
:100C3000FE010E94F429C93FD107C9F70E94481854
:100C40000C94312ADDC9E8E5F3E0A0E0B8E00080CB
:100C50000EBC8111012C1197A0FDFDCF0192B9F7B7
:100C60000DB40895B0E0A0E0E8E3F6E00C94FE29AE
:100C700030E0F901E80FF91F1E161F060CF07AC0CC
:100C8000803891050CF076C0802E912CD401A60FEF
:100C9000B71F1A161B060CF06DC0603471050CF0FE
:100CA00069C0E62FE7707E2EE7E08E0E911CE3E030
:100CB00095948794EA95E1F7F3E075956795FA9531
:100CC000E1F7062E000C770BDB01B695BA2FAA27A9
:100CD000B795A795A80FB91FA85ABC4FEA01F12CE8
:100CE000E12C6701C60ED71E48E0C416D1040CF0F3
:100CF00041C0EFEFCE16DE0694F18C0150E040E0EB
:100D000017FD23C0FA01EC0FFD1FA490B12C072C96
:100D100002C0AA0CBB1C0A94E2F7EFEFCE16DE0667
:100D200071F1FD01E40FF51F60806A286082772071
:100D300061F0E7E0CE16D10441F0FD01E058FF4F2D
:100D4000E40FF51FA080BA28B0824F5F5F4F0F5F9E
:100D50001F4F421753071CF40038110589F64FEF57
:100D6000E41AF40AA058BF4FC20FD31F8E149F0479
:100D700009F0B7CFCDB7DEB7EEE00C941A2A7110A8
:100D8000DCCFE3CF90915703911103C08FEF9FEF1A
:100D900008954FB7F89422E02093E9005091F200B3
:100DA000252F30E01216130614F421E030E0232B37
:100DB00031F0289884E6809356038091F100552302
:100DC00039F03091F200311103C06BE66093E80016
:100DD0004FBF5523D9F290E008952FB7F89483E0E0
:100DE0008093E9009091E800892F807295FF04C0FC
:100DF0003091F20080E4831B2FBF089580914E0351
:100E000081110DC022E020934A0334E030934B035C
:100E100010924D0310924C0341E040934E038AE43C
:100E200093E00895FC0110D0319728F068517C4F71
:100E30008F4F9F4FF9CFAB01FC0106D064177507A8
:100E40008E079F07D0F30895A6E4B3E02FB7F89478
:100E50007D918D919C9166B52FBFA89B05C06F3F7A
:100E600018F47F5F8F4F9F4F22E0660F771F881F18
:100E7000991F2A95D1F70895409154025091550237
:100E8000209152023091530242175307B4F49091CB
:100E9000E8009570E1F33091E80032FD19C08093CD
:100EA000F100809154029091550201968F73992719
:100EB000892B19F45EEF5093E800A0915402B09191
:100EC00055021196B0935502A093540281E0089503
:100ED00080E00895B0E0A0E0E0E7F7E00C94052A98
:100EE000D82E8A01EB017B01E40EF51ECE15DF053D
:100EF00051F0D7FE0EC0FE018491BEDF2196811114
:100F0000F5CF0FEF1FEFC801CDB7DEB7E7E00C94C8
:100F1000212A8881F2CFA1E0B0E0E1E9F7E00C946A
:100F2000082A82E0898342E450E06EEE77E080E8B0
:100F3000D1DF64DFFC01028113810115110589F005
:100F4000D801ED91FC910280F381E02DBE016F5F2D
:100F50007F4FC801099597FD04C0F80100851185F0
:100F6000ECCF89812196E4E00C94242A615030F082
:100F70002091F100FC0120830196F8CF289884E6A7
:100F8000809356030895B0E0A0E0E9ECF7E00C94FC
:100F9000022A6C017B018B01040F151FEB015E011E
:100FA000AE18BF08C017D10759F06991D601ED916D
:100FB000FC910190F081E02DC6010995892B79F70C
:100FC000C501CDB7DEB7EAE00C941E2AB0E0A0E080
:100FD000ECEEF7E00C94022A6C01B62EA72E7A01F3
:100FE00080910B01882309F453C0209157032223D9
:100FF00009F44EC00091580200FF05C01091E000B6
:1010000012601093E000E70110E00AEF209711F45E
:101010001123B9F1E2DE811106C00150C9F181E06E
:1010200090E000DFF3CF8C171D0611F00CF08C2F31
:101030009FB7F89433E03093E9004091E80045FD14
:1010400002C09FBFE3CFC81BD109EB2DFA2DBE2EE6
:10105000AF2E815020F0A190A092F100F8CF112383
:1010600029F07AE37093E80010E0EBCF5091E800AC
:1010700055FDE7CF6AE36093E80011E0209709F39C
:10108000F3CF5D98A4E6A09357021E141F043CF012
:10109000C1E0D0E0F601D383C283F12CE12CC7017B
:1010A000CDB7DEB7EAE00C941E2AA1E0B0E0EBE594
:1010B000F8E00C940A2A6983DC01ED91FC9102802E
:1010C000F381E02D41E050E0BE016F5F7F4F099555
:1010D0002196E2E00C94262A83E08093E900209197
:1010E000F200222319F03AE33093E800089575DE08
:1010F00090E00895FC018485958597FD05C02FEF4C
:101100003FEF3587248708953DCE0895CF93DF9331
:10111000EC018C859D8597FF03C034DE9D878C870D
:101120008C859D85DF91CF910895FC0184859585FF
:1011300097FD0BC03FB7F89442E04093E9008091DF
:10114000F2003FBF90E0019608959FB7F89422E027
:101150002093E9008091F2009FBF90E0089590E015
:1011600061CE08958FB18095807F669B88601C9BBF
:1011700084600895CF93C82FF5DF982F9C2381E0DA
:101180009C1380E0CF91089580E05DCD0895603498
:101190007105D0F5480F592F511D41155105A1F189
:1011A000803891058CF54138510514F040E850E045
:1011B000481BFB0133E0F595E7953A95E1F7F69585
:1011C000FE2FEE27F795E795E80FF91FE85AFC4F39
:1011D0006770772781E090E001C0880F6A95EAF791
:1011E000382F213041F4415078F08191DF0111977F
:1011F000832B8C93F8CF8095415030F09191DF0193
:10120000119798239C93F8CF089580389105B8F4EE
:1012100060347105A0F490E121E061FD24E060FDFF
:10122000220F62FD2295687F969FD0011124A80F9E
:10123000A85ABC4F0C90022A40FF02260C92089537
:10124000B0E0A0E0E6E2F9E00C94002A6D3089F00D
:10125000C0902903D0902A036A3091F410922C0395
:1012600010922B0388E0C80ED11CD0922A03C092A2
:10127000290381E090E0CDB7DEB7ECE00C941C2AA6
:1012800000912B0310912C03E5E06E9FE0011124E7
:10129000C251DD4F4801F12CF5E0E12CFF1629F099
:1012A000CE010196FE01E490EC01B12CA12C4E2D53
:1012B0004170B6016A0D7B1DC401A7DFE694FFEF04
:1012C000AF1ABF0A88E0A816B10489F7F394EFEFCC
:1012D0008E1A9E0A26E0F212DFCF0A5F1F4F10938C
:1012E0002C0300932B03C5CF0F931F93CF93DF9352
:1012F0008C01D0E0C0E0F801EC0FFD1F6491662383
:1013000039F088EA97E09CDF892B11F02196F3CF22
:10131000CE01DF91CF911F910F910895B0E0A0E031
:10132000E4E9F9E00C94052A7C01D22E8B01040F2C
:10133000111DEB0177FF02C0D0E0C0E0C80101340D
:10134000110514F080E490E0C817D90734F44D2D4E
:10135000BE01C7015ADF2196F1CFCDB7DEB7E7E076
:101360000C94212AB0E0A0E0E8EBF9E00C94032A09
:101370007C016B01B42E122FEC01C7018B0D911D66
:10138000C817D9073CF4202F412FB601CE01C6DF84
:101390002196F3CFCDB7DEB7E9E00C941F2ACF92A8
:1013A000DF92EF92FF920F93CF93DF936C017B015B
:1013B000C42FD22F202FEBDEB7016D0F711D6150AE
:1013C0007109202F4C2FC601E2DE202F4D2FB701CF
:1013D000C601A4DFC6018C0F911D202F4D2FB70130
:1013E00001979CDFDF91CF910F91FF90EF90DF90FD
:1013F000CF9008950F9300E128E54EE352E0BC0141
:1014000084E190E02FDC0F910895262F30E043E037
:10141000849FC0011124EEE2F3E067E070E0082E43
:1014200002C0660F771F0A94E2F7609570954485B5
:1014300055856423752302C0220F331F8A95E2F776
:10144000622B732B758764870895FC019481492F63
:1014500050E0559547955595479543704F5F4430FB
:1014600009F441E0937F84E0489F90011124292BE7
:101470002483089598E0699FB0011124E82FE69530
:10148000E60FF72FF11DEE5AFE4F908180FD08C048
:101490009F7080E1489FA0011124942B90830895B0
:1014A000907F492B40830895982F70E0FB01EE0F49
:1014B000FF1FE053FD4F21E030E0082E02C0220F55
:1014C000331F0A94E2F74081518124233523232BD3
:1014D00089F4E82FE695F0E083E0660F771F8A95A0
:1014E000E1F7EE5AFE4FE60FF71F808190FF8295DD
:1014F0008F70089580E008951F93CF93DF93182F86
:10150000EB01888190E02A812223F1F043E050E052
:10151000840F951F23E0959587952A95E1F7809391
:101520001003612F70E0685F7F4F33E0759567951A
:101530003A95E1F760932D03B7DF811108C0198355
:10154000DF91CF911F91089541E050E0E1CF81E01C
:10155000F7CF0F931F93CF938C01FC018381C1813F
:10156000CD5FC81BC83008F4C8E0181694F0F80125
:101570001382B8018C2FC0DF8130C1F4B8018FEF26
:101580008C0FBADF813091F4B8018EEF8C0FB4DF8D
:101590000DC08150F801838384305CF3B8018C2F37
:1015A000ABDF813019F423E0F8012383CF911F9141
:1015B0000F91089580913103843038F560912F03A5
:1015C000611101C061E080912E0390E02091300311
:1015D0002223E1F043E050E0840F951F23E095952E
:1015E00087952A95E1F78093100370E0675F7F4F3E
:1015F00033E0759567953A95E1F760932D0354DFD5
:10160000882319F038E030933103089541E050E029
:10161000E3CF8F30B8F48F5FE62FF0E0EE0FFF1FBF
:10162000E053FD4F21E030E0082E02C0220F331FAF
:101630000A94E2F74081518124233523232B11F4AE
:1016400033CF089580E008958823C1F08150E62FBC
:10165000F0E0EE0FFF1FE053FD4F21E030E0082ED9
:1016600002C0220F331F0A94E2F7408151812423E4
:101670003523232B11F418CF089580E00895CF93DC
:10168000DF93FC01EB0190912E039695969596952C
:10169000809130038130B1F59150908360912F0398
:1016A00070E06C5F7F4FE3E075956795EA95E1F731
:1016B000688380912E0390E00296F3E095958795DC
:1016C000FA95E1F7C1DF382F377FC9F460912F0316
:1016D00070E0645F7F4F53E0759567955A95E1F729
:1016E000688380912E0390E0029673E0959587952C
:1016F0007A95E1F7A9DF482F477F09F480E0DF9171
:10170000CF9108959F5F908360912F0370E06C5F8D
:101710007F4F33E0759567953A95E1F7688380913F
:101720002E0390E0029643E0959587954A95E1F760
:1017300070DF282F277F19F760912F0370E0645F17
:101740007F4F83E0759567958A95E1F7688380916F
:101750002E0390E0029623E0959587952A95E1F770
:1017600058DFC9CFCF93DF93FC01EB0190912E039B
:1017700080913003813009F05AC0983008F455C088
:101780009695969596959150908360912F0370E071
:10179000645F7F4F83E0759567958A95E1F768836D
:1017A00080912E0390E0029623E0959587952A95E7
:1017B000E1F74ADF811105C031E0832FDF91CF913E
:1017C000089560912F0370E06C5F7F4FA3E07595E3
:1017D0006795AA95E1F7688380912E0390E00296C1
:1017E000B3E095958795BA95E1F72EDF882321F32D
:1017F00080912F0390E0BC016450710977FF02C013
:10180000695F7F4FE3E075956795EA95E1F7688337
:1018100080912E0390E00296F3E095958795FA95D6
:10182000E1F712DF31E0882341F230E0C6CF28E84B
:10183000290F2830D0F39695969596959F5F9083C3
:1018400060912F0370E0645F7F4F53E0759567955B
:101850005A95E1F7688380912E0390E0029673E039
:10186000959587957A95E1F7D4DE882309F4A4CF7E
:1018700060912F0370E06C5F7F4F33E07595679543
:101880003A95E1F7688380912E0390E0029643E059
:10189000959587954A95E1F7BCDE882309F48CCFAE
:1018A00080912F0390E0BC016450710977FF02C062
:1018B000695F7F4F83E0759567958A95E1F7688347
:1018C00080912E0390E0029623E0959587952A95C6
:1018D000E1F79FDEA7CFE82FF0E0E95EFC4F8081C3
:1018E000982F9770FB01908386958695869590E05A
:1018F0000895EF92FF921F93CF93DF931F92CDB77E
:10190000DEB7982F969596959695E92EF12C9F50D7
:101910009430F0F4482F477013E0419FA001112448
:1019200020913A0330913B0302C0369527954A95A2
:10193000E2F72770B7016F5071092617170641F4B7
:1019400081E00F90DF91CF911F91FF90EF9008956C
:10195000182F1982BE016F5F7F4F80E0BCDF8E15AC
:101960009F0529F42981812F8770281748F7BE0128
:101970006F5F7F4F81E0AFDF8E159F0529F43981BE
:10198000512F57703517E0F6BE016F5F7F4F82E031
:10199000A2DF8E159F0529F47981A12FA7707A17F0
:1019A00078F6BE016F5F7F4F83E095DF8E159F0550
:1019B00031F4B981E12FE770BE1708F0C1CFBE0145
:1019C0006F5F7F4F84E087DF8E159F0531F4F981CB
:1019D000912F9770F91708F0B3CFBE016F5F7F4F5B
:1019E00085E079DF8E159F0531F44981612F67709D
:1019F000461708F0A5CFBE016F5F7F4F86E06BDF13
:101A00008E159F0531F42981812F8770281708F0E2
:101A100097CFBE016F5F7F4F87E05DDF8E159F051B
:101A200031F43981512F5770351708F089CFBE0135
:101A30006F5F7F4F88E04FDF8E159F0531F479810E
:101A4000A12FA7707A1708F07BCFBE016F5F7F4F81
:101A500089E041DF8E159F0531F4B981E12FE770F0
:101A6000BE1708F06DCFBE016F5F7F4F8AE033DF96
:101A70008E159F0531F4F981912F9770F91708F0B1
:101A80005FCFBE016F5F7F4F8BE025DF8E159F0517
:101A900031F44981612F6770461708F051CFBE01BC
:101AA0006F5F7F4F8CE017DF8E159F0531F4298122
:101AB000812F8770281708F043CFBE016F5F7F4FDB
:101AC0008DE009DF8E159F0531F43981512F577054
:101AD000351708F035CFBE016F5F7F4F8EE0FBDE1C
:101AE0008E159F0531F47981A12FA7707A1708F020
:101AF00027CFBE016F5F7F4F8FE0EDDE8E159F0514
:101B000029F41770E980E11608F01ACF80E019CFA8
:101B1000A1E0B0E0EEE8FDE00C94062A7C01062F7F
:101B200010E0BE016F5F7F4F812FD5DE9C018E15C7
:101B30009F0511F599819923F9F0E12FF0E0E95E15
:101B4000FC4F091758F4901B9770EE0CEE0CEE0C3E
:101B50009E2990832196E6E00C94222A10821F3061
:101B600020F4818181931F5FFACF10922603602FAA
:101B7000691BC901CDDFEECF1F5F103191F6EACFAF
:101B8000A1E0B0E0E6ECFDE00C94062A7C01062F13
:101B900010E0BE016F5F7F4F812F9DDE8E159F0588
:101BA00011F0892B09F569816730F0F4E12FF0E03D
:101BB0008E2D880F880F880FE95EFC4F462F400F4F
:101BC0005527551F4830510544F4600F6770682B46
:101BD00060832196E6E00C94222A87608083075078
:101BE000600FC701CDDFF5CF1F5F103191F6F1CF48
:101BF000B0E0A0E0EEEFFDE00C94052A182FC0E065
:101C000048E0612F8C2F36DCDD24D394D10E40E0E8
:101C10006D2D8C2F2FDC02E0010F40E0602F8C2F08
:101C200029DC83E0E82EE10E40E06E2D8C2F22DCD3
:101C300094E0F92EF10E40E06F2D8C2F1BDCD5E0E7
:101C4000D10F48E06D2F8C2F15DCCF5FC031C1F66E
:101C500040E0612F80E00EDC40E06D2F80E00ADC88
:101C600040E06D2F81E006DC48E06D2D82E002DC73
:101C700048E0602F82E0FEDB48E06E2D82E0FADB78
:101C800043E06F2D82E0F6DB4CE0602F86E0F2DB74
:101C900043E06D2D87E0EEDB48E0602F87E0EADB74
:101CA00048E06E2D87E0E6DB48E06F2D87E0E2DB61
:101CB00043E06D2D8CE0DEDB48E0602F8CE0DADB6A
:101CC00048E06E2D8CE0D6DB48E06F2D8CE0D2DB57
:101CD00040E06D2F8AE0CEDB40E06D2F8BE0CADB69
:101CE0004CE06E2D8BE0C6DB4CE0602F8FE0C2DB5A
:101CF0004DE06F2D8FE0BEDB40E06D2F8FE0BADB53
:101D000040E06D2F8EE0B6DBCDB7DEB7E7E00C9498
:101D1000212ACF93DF9384E08093CF0221E02093A8
:101D20003E0320933D0393E294BD3FEF38BD41EF66
:101D3000409380001092880010928A00CEE2D3E097
:101D4000298758EC5A87E7E1F3E01082118212826A
:101D500013821482158216821782108611861286CB
:101D6000138614861586168617861D861C86DF91B7
:101D7000CF910895089590E080E00895BF920F9369
:101D80001F93CF93DF93CDB7DEB7A1970FB6F8942B
:101D9000DEBF0FBECDBFB42E19A221E0241710F074
:101DA0002AE0B22E8E010F5D1F4F2B2D30E050E048
:101DB00040E00E948329E62FB901CA01EA302CF5E0
:101DC000E05DD801EE938D01232B242B252B69F7A1
:101DD00090E080E0109769F0FD0101900020E9F7A4
:101DE000AF01415051094A1B5B0BBD0188EA97E0E6
:101DF000CAD8A1960FB6F894DEBF0FBECDBFDF9153
:101E0000CF911F910F91BF900895E95CDACFFC014B
:101E100001900020E9F7AF0141505109481B590BCF
:101E2000BC0188EA97E0AFC80895682F70E090E0A1
:101E300080E04AE0A3CF0895EF92FF920F931F93A3
:101E4000CF93DF9388E096D9882309F474C009E71B
:101E50000093100310922C0310922B0310922A036C
:101E60001092290382EE90E03FDA10922C03109238
:101E70002B038CE0E82EF12CF0922A03E092290348
:101E80001091370310932D038AED90E02DDAC4E210
:101E9000D0E0D0932C03C0932B03F0922A03E0925E
:101EA0002903812FC2DF10922C0310922B0308E12B
:101EB00010E010932A030093290382ED90E014DAD6
:101EC0008091390386958695869580932D03D093CE
:101ED0002C03C0932B0310932A0300932903A5DF3F
:101EE00010922C0310922B03D0932A03C093290342
:101EF0008AEC90E0F9D980913903877080932D03A3
:101F0000D0932C03C0932B03D0932A03C0932903AF
:101F10008CDF10922C0310922B0320E330E03093DF
:101F20002A032093290389EB90E0DED9CDB7DEB7F1
:101F3000E6E00C94222A80911003893709F08ACFB9
:101F400011D983FD87CFE5DE1092100383CFB0E077
:101F5000A0E0EDEAFFE00C94FC29882E162F542E09
:101F6000422E8AE0689F700111248AE2E80EF11C7B
:101F7000E60EF11C01E02AE047E7B70181E090E0BE
:101F80000EDA912CF401EB5EF64FA490B12C93E0A5
:101F9000B594A7949A95E1F7D491D12CC12C2D2F0B
:101FA0002770C21608F0D1C0F401EA5EF64FEC0DBE
:101FB000FD1DC49146E050E050932C0340932B0349
:101FC000D7011196B0932A03A0932903EA2DED318E
:101FD00008F025C0F0E0E151F04F0C94F4290C100A
:101FE0005110541057105A105D1060106310661095
:101FF00069106C106F107210751078107B107E10C5
:102000008110841087108A108D10901093109610F4
:1020100099109C109F10A21083E392E065D937E0DD
:102020003415D8F151E05515C0F5111136C04C2FBB
:1020300046954695469561EF640F643070F18CE1EA
:102040008C9D30018D9D700C11244150550B83E007
:10205000440F551F8A95E1F74557564F08E028E091
:1020600061E270E0C30103960E9432068EE0680EC2
:10207000711C70922C0360922B0381E290E090938C
:102080002A03809329038AE391E0C1DEC7706C2F95
:1020900070E090E080E04AE071DE8FEFC81AD80A65
:1020A0007ECF86E292E0BACF8BE192E0B7CF8EE0AE
:1020B00092E0B4CF88E092E0B1CF80E092E0AECF82
:1020C00089EF91E0ABCF8EEE91E0A8CF83EE91E067
:1020D000A5CF87ED91E0A2CF87EC91E09FCF89EB70
:1020E00091E09CCF8FEA91E099CF84EA91E096CF7E
:1020F00085E991E093CF88E891E090CF8DE791E07A
:102100008DCF81E791E08ACF81E691E087CF83E5AB
:1021100091E084CF88E491E081CF8CE391E07ECFA1
:102120008CE291E07BCF8DE191E078CF82E191E08C
:1021300075CF86E091E072CF8FEF90E06FCF86EFA2
:1021400090E06CCF8CEE90E069CFCDB7DEB7E0E1E8
:102150000C94182ACF931092320388E080933303B3
:10216000C0E020911103C21708F08AC04C2F50E044
:1021700036E0C39FF0011124ED59FD4F958199235D
:1021800009F464C0218180912F03281B022E000CCA
:10219000330B37FF03C031952195310925303105C7
:1021A0000CF054C066E0649FF001659FF00D1124AF
:1021B000ED59FD4F208170912E03A22FA71B809116
:1021C0003B038695869586958E708F5F6091300370
:1021D00061113EC0AE3FA4F0A63094F4A92FA81B15
:1021E000BB0B129714F0692F681B96E0949FF001C7
:1021F000959FF00D1124ED59FD4F65832C5F2083D1
:1022000086E0849FF001859FF00D1124ED59FD4F6C
:10221000458141111BC00E94832864E670E00E9442
:10222000E1294E9724F461E08DE090E0A9DC509123
:102230003903252F2695269526952F5FF8E02F9FA9
:10224000900111245770522B50933903CF5F89CFDF
:102250006130B1F6A330A4F6AB3F94F2E92FE81B4E
:10226000FF0B981B32970CF490E0B6E0B49FF0019E
:10227000B59FF00D1124ED59FD4F95832450BFCF2C
:10228000CF91089580E40E94BA08882321F022E0CB
:1022900020933303089580E20E94BA088111F7CF9A
:1022A00080E80E94BA08882311F084C9089580E16B
:1022B0000E94BA08882391F030913503311126C06D
:1022C00043E040933503509134035F5F543019F07D
:1022D00050933403089510923403089584E00E94CB
:1022E000BA08882311F036CF089588E00E94BA0812
:1022F00010923203882351F080913303843021F00F
:10230000813011F01092360324E0C2CF0895CF93AC
:10231000C82F809132038F5F63E00E94C0299093A1
:102320003203911104C081E080933303ABDF88E076
:102330000E94BA08882339F0209136032F5F2C17AA
:1023400058F4209336030E94B208982F987083FDAA
:1023500009C01092360303C01092360391E0892F12
:10236000CF91089590E0FBCF90913B03835097FF6E
:10237000B1C028E220933F0330E43093900040EA5C
:1023800057E050939900409398008B3008F097C025
:10239000E82FF0E0E253FE4E0C94F429D911F51128
:1023A000F011FD11F9115F125F12011205124812AE
:1023B0005A1297FF0CC0F8E2F0933F0390E4909319
:1023C000900021E43FE030939900209398003091F1
:1023D00012033F5F303408F03FE330931203089557
:1023E00061E085E090E0CCCB089561E081E090E091
:1023F000FACF61E082E090E0F6CF61E084E090E027
:10240000F2CF61E083E090E0EECF61E08EE090E01B
:10241000B7DB0E94832864E670E00E94E1298233E2
:10242000E8F463E081E090E0ABDB61E084E090E021
:10243000A7DB61E08DE090E0A3DB70913B0377FFC9
:102440005CC0B8E2B0933F03E0E4E093900063E641
:1024500070E070939900609398000895803560F45F
:1024600062E08AE090E08CDB62E083E090E088DB71
:1024700062E084E090E0E0CF61E08EE090E080DB1D
:1024800062E08CE090E07CDB62E08BE090E0D4CF17
:1024900097FF0CC058E250933F0360E460939000B4
:1024A000A2E5B0E0B0939900A093980061E08AE0C3
:1024B00090E099CF809139038F5F8093390397FF24
:1024C0001CC048E240933F0380E48093900061E4A5
:1024D0007FE0BFCF8B3088F4E82FF0E0EE58FD4E60
:1024E0000C94F429D911F511F011FD11F9117D1297
:1024F0007D120112051248125A1208950F931F936C
:10250000CF93DF93C82FD62F142F022F112391F1D1
:102510008EEF8C0F8D3070F5DD3160F56D2F8C2FC7
:102520000E94540A882331F1402F6D2F8C2F0E9476
:102530003A0A1130F9F00E9483286CE070E00E94A2
:10254000E12980932D0311508B3070F0202F412F03
:102550006D2F8FEF8C0FD2DF202F412F61E06D0F99
:102560008C2FCCDFCF5FD2CF8830B0F78630D0F35E
:10257000DF5FCCCFDF91CF911F910F9108951F9313
:10258000CF93DF93C82FD62F142F112309F47AC0CD
:102590008EEF8C0F8D3008F075C0DD3108F072C001
:1025A0006D2F8C2F0E94540A882309F46BC040E0E1
:1025B0006D2F8C2F0E943A0A0E94832864E670E0F7
:1025C0000E94E129482F80932D0390911103292F18
:1025D00030E0A09137035A2F5695569556956FE0E7
:1025E00070E0651B7109261737076CF5413558F106
:1025F00076E0729FF001739FF00D1124ED59FD4FAD
:10260000BC2FBB0FBB0FBB0FB0838D2F880F880F64
:10261000880F8183128253E05383A695A65FA5831A
:10262000A1E04E3520F4A2E0473508F4A3E046E0EF
:10263000429FF001439FF00D1124ED59FD4FA483FB
:102640009F5F909311031130E9F00E9483286CE0A2
:1026500070E00E94E12980932D0311508B3060F0CF
:10266000412F6D2F8FEF8C0F8ADF412F61E06D0FAF
:102670008C2F85DFCF5F89CF8830B8F78630D0F3D5
:10268000DF5F83CFDF91CF911F9108950C942F29A5
:10269000089582E090E0FADF882319F03E9A579A75
:1026A00008953E98579808950F931F93CF93DF9303
:1026B0008FEF90E0EBDF8E3B59F080E091E0E6DFBA
:1026C000893731F081E091E0E1DF813009F044C0E9
:1026D00082E091E0DBDF8093370383E091E0D6DF97
:1026E0008093380310923B0310923A0384E091E008
:1026F000CDDFC82FD0E0DC2FCC27D0933B03C09395
:102700003A0385E091E0C2DFC82BD0933B03C0932E
:102710003A0386E091E0BADF8093390307E113E0E2
:10272000C7E0D1E0CE01B2DFF80181938F0121969D
:10273000C731F1E0DF07B1F783E284BD18BC11EFC8
:10274000109380001092880010928A0081E0DF913F
:10275000CF911F910F91089580E0F9CF1F93CF93F0
:10276000DF93EC01162F0E942F29181721F0612FFB
:10277000CE010E944929DF91CF911F9108950F93B7
:102780001F93CF93DF9381EC80937C0001E705B921
:1027900017E614B925E32BB93FE33AB9769A6E9858
:1027A00040EF41BB10BA50E55CBD61E06DBD85E016
:1027B0000E94AF08599A85E00E94AF085C98ECEA45
:1027C000F0E075917EBD00000DB407FEFDCFE93B42
:1027D000C1F75C9A91E890936400A1E0A093650032
:1027E0000E94C40880E80E94BA088823A9F05C9877
:1027F000B5EABEBD00000DB407FEFDCF5C9A2E9871
:1028000058982D98C0916400C062C0936400D1E0D4
:10281000D3BF889513BEFBCF84E00E94BA088823FB
:10282000B9F12D9884E80E94BA088823A1F02D9A66
:1028300088EC0E94AF0858986FEF82E090E00E9409
:10284000372984EF91E00E941207589A84E80E9489
:10285000BA088111FBCF84E10E94BA088823A1F055
:102860002D9A88EC0E94AF082E9860E082E090E0FC
:102870000E94372984EF91E00E9412072E9A84E18A
:102880000E94BA088111FBCF88EC0E94AF08C4CF28
:102890002D9AFFDE81E090E00E942F2981FF0EC07B
:1028A000082F047082FD2E98C1EFDFEF80E40E94B4
:1028B000BA08882309F464C02E9A589A82E30E94C9
:1028C000AF080E94B2088111F9CF10922D03109227
:1028D0003C031092CF021092100388E280930C0107
:1028E000109164001E7F1093640030917A00306470
:1028F00030937A0050917A0056FDFCCF0091780019
:10290000109179000E942407AB01BC01C801B0E01E
:10291000A0E0DC01992788278C019D01040F151F79
:10292000261F371FC901B801E0916400E160E09300
:102930006400611571058105910511F00E94262939
:102940000E9424076093130370931403809315036C
:1029500090931603DED910923B0310923A036FEF67
:102960007FEF709365076093640793DE1092900089
:102970007AE070939100DF91CF911F910F910895AC
:10298000002329F0C430D10511F42E9A589881E023
:102990000E942306CE010E94FA090E94C4088FE01B
:1029A0000E94AF082196C931D10509F07FCF0023DD
:1029B00011F0589A2D9880E991E00E9412072D9A03
:1029C00081E090E00E942F2980FF78CF8AE090E09C
:1029D0000E942F29FFEFF80FFE3F08F06FCF22E390
:1029E00030E030932C0320932B0348E350E05093C6
:1029F0002A0340932903CAE0D0E0682F88EA97E0D1
:102A00000E9420092196CE010E942F29C031D105B4
:102A1000A1F70E94C40888EE93E00E9412074ECFEF
:102A20000F920FB68F939F93EF93FF938091410383
:102A30008D5F8D3708F08D5780934103E2E4F3E01A
:102A400080818E4F808391819F4F918382818F4FB0
:102A5000828383818F4F8383E6E4F3E080818F5FFD
:102A6000808381818F4F818382818F4F8283838195
:102A70008F4F83838FB18F6066991C9B88278F3619
:102A800081F480914003981B963068F0E0E0F8E014
:102A900087E78083818388E180936000F093600002
:102AA000FFCF90934003FF91EF919F918F910FBEC5
:102AB0000F9018951F920F920FB60F9211248F93BB
:102AC0009F938091E1009091E100937F9093E100CA
:102AD00083FF0FC01092E90091E09093EB001092F9
:102AE000EC0092E39093ED001092570398E09093DE
:102AF000F00082FF22C093E09093E9009091F200F1
:102B0000992319F09AE39093E80090915702992342
:102B100041F090915702915090935702911101C04A
:102B20005D9A90915603992341F0909156039150EC
:102B300090935603911101C0289A84FF18C0909178
:102B4000E2009E7E91609093E2008091E1008F7E92
:102B50008093E100809158028E7E806180935802BC
:102B60009F918F910F900FBE0F901F90189580FF2F
:102B7000F7CF8091E2008E7E80618093E200909199
:102B8000E1009E7E9093E100809158028E7E8160EC
:102B9000E5CF1F920F920FB60F921124CF92DF92C2
:102BA000EF92FF920F931F932F933F934F935F9357
:102BB0006F937F938F939F93AF93BF93EF93FF9305
:102BC000CF93DF93CDB7DEB76C97DEBFCDBF10924A
:102BD000E9008091E80083FF25C068E0CE014596BA
:102BE0000E94B60702EF0093E8001D8917FF39C065
:102BF000C090E800C0FEFCCF212F207609F032C142
:102C00003E894F89588D6F89F88C311131C0103849
:102C100061F5F0905902F092F1001092F100FEEF90
:102C2000F093E8006C960FB6F894DEBF0FBECDBFF0
:102C3000DF91CF91FF91EF91BF91AF919F918F91D4
:102C40007F916F915F914F913F912F911F910F91C4
:102C5000FF90EF90DF90CF900F900FBE0F901F90DE
:102C600018959EEF9093E800C7CF1092F100D5CF52
:102C7000313059F41111D3CF4130510581F6809193
:102C800059028D7F80935902CACF333049F4111114
:102C9000C6CF4130510519F6809159028260F2CFBA
:102CA000353041F4D090E800D0FEFCCF60686093EE
:102CB000E300B5CF363009F0A7C00B8D1C8D92E034
:102CC0001092E9001092550210925402F9122EC08F
:102CD00010925302109252020E948B071F8259E0F9
:102CE0005983FA8271E07E83B0EAB8872AEF298798
:102CF0004091540250915502475F5F4F5C834B8374
:102D00008D831092E9001092550210925402109394
:102D100053020093520249E050E0BE016F5F7F4FC3
:102D200080E00E946A070E948B0779CF10935302BC
:102D3000009352020E94FE06FC01C280D380C1149F
:102D4000D10409F451C1D601ED91FC910480F581C3
:102D5000E02DBE016B5E7F4FC6010995009709F01B
:102D60003EC1F601C084D184EACF33E0F3120DC036
:102D70004F89442309F43FC0423059F440E867E0EA
:102D800082E598E037D181114ACF61E26093EB0090
:102D900049CF413029F440E86BE086E498E0F2CF77
:102DA000433099F70E94FE06FC01C280D3808E0159
:102DB0000F5F1F4F7801C114D10479F0D601ED9156
:102DC000FC910680F781E02DB801C6010995080F36
:102DD000111DF601C084D184EECFD8011C92F701F9
:102DE00001900020E9F7BF01615071096E197F0958
:102DF00040E0C701C7CF60E378E0FB01449150E0B9
:102E000080E80E946A070BCF373009F4BECF383014
:102E100021F4F1E0F093F10002CF393009F0FFCE58
:102E2000137009F0B2CFE6E1F1E081E05191552352
:102E300081F08093E90071E07093EB00DF0111975E
:102E4000CC90C092EC00B6E3B093ED008F5F87307A
:102E500069F72EE72093EA001092EA00EF88E092EB
:102E60005703DDCEEB8CFC8C1092E90010925502DA
:102E700010925402F0925302E0925202D98CD11077
:102E800094C03E894D89413A49F4313209F07DCFF1
:102E900047E050E064E071E080E0B3CF413209F0F8
:102EA00074CF333269F48F89988DB0E0A0E08093BD
:102EB000000190930101A0930201B0930301AFCEF2
:102EC000303269F4D090E800D2FEFCCF67E084E0B5
:102ED00091E00E94B6070BEF0093E800A0CE3232DB
:102EE00009F09DCEFF88F0920B01EEEFFFE76591B0
:102EF00074916B3F7C4D51F1E0E0F8E0809104016A
:102F000090910501A0910601B0910701803B94408A
:102F1000A105B105F1F450910B0150FD1AC0EE3F2F
:102F20008AE0F80791F5A7E7B7E7B183A083F091AE
:102F30006000F093560218E19BE00FB6F894A89554
:102F4000109360000FBE9093600069CEEEEFFAE040
:102F5000D5CFC080D180A7E7CA16DA0609F05FCEC8
:102F6000A89570916000786170936000B0915602EE
:102F7000B0936000EE3F2AE0F20791F02091FE0A44
:102F80003091FF0A318320834ACEE080F180B7E799
:102F9000EB16FB0641F2F092FF0AE092FE0AC3CF65
:102FA0001092FF0A1092FE0A3ACE0E94FE06FC0121
:102FB000028113810115110509F4E7CED801ED91C5
:102FC000FC910190F081E02DBE016B5E7F4FC80146
:102FD0000995811124CEF80100851185EBCF1816D3
:102FE00019060CF41CCED1CE11E0F112BECE64E372
:102FF00078E003CFEF92FF920F931F93CF93DF936D
:10300000F82E192FE62E042F81E0860F880F0E94DC
:103010003C0783E00E943C07CF2DD12FEC0EFD2E04
:10302000F11CCE15DF05A9F007FF11C0FE01849148
:103030000E943C07182F80E00E943C0781232196C4
:103040008111EFCFCDB7DEB7E6E00C94222A88815C
:10305000EFCF81E0F7CFE8E5F7E01382128288EE48
:1030600093E0A0E0B0E084839583A683B78380E2F9
:1030700091E0918380838FEF9FEF95878487E8EAC3
:10308000F7E01382128282E391E0918380830895B6
:1030900000D01F92CDB7DEB7789483E084BD83E083
:1030A00085BD81E080936E00E1E8F0E083E08083FD
:1030B000E0E881E08083E1E983E08083E0E981E08A
:1030C0008083E1EC87E08083E3EC81E08083E0ECC7
:1030D00082E08083E2EC81E08083EAE787E080831E
:1030E0008068808310925703109259021092580200
:1030F0000091D70001600093D70010EA1093D80028
:1031000029B5206129BD39B5326039BD39B4432DA7
:1031100041704B8330FEFACF81E090E00E941207AD
:103120005091D8005F7C50615093D8006091E000CE
:10313000607F6093E0007091E1007E7E7093E1001B
:103140009DE09093E200559A209A19DBA0915A02D3
:10315000AA2349F010925A0280E090E0892BB1F343
:103160000E940000F3CF4090420350905B02842DF8
:103170008519B82F60900C01861540F4BF5FB61515
:1031800058F751E053BF889513BEE6CFE1E0E093D6
:103190005A0240925B02E7E2F3E08081918101965E
:1031A00080839183E8E5F3E0A111AFEF8FEFA19366
:1031B000A193A193A1938150D0F710922A0310926A
:1031C000290310922C0310922B03F0913F03FF234D
:1031D00059F0F150F0933F03F11108C010929000A4
:1031E00070903F03711002C010929000F0903E0367
:1031F00001E0F0123AC08090130390901403A09065
:103200001503B0901603C501B40120E23EE440E08E
:1032100050E00E945729675B744FDB01CC908C0C07
:10322000911CA11CB11C8092130390921403A092D4
:103230001503B09216031091CF021F5F212F153096
:1032400008F024E02093CF0288E00E94BA08882387
:1032500009F417C180903D0380FEF2C010923D0337
:1032600043E040933E0310923C0350913E035430A0
:1032700011F40E941C0F70913E03723009F0A7C632
:10328000D09033039D2D9071592ED4FE44C780E811
:103290000E94BA08882379F06091350360FD0BC065
:1032A0003091CF02311101C031E031503093CF0263
:1032B00061606093350380E10E94BA08882361F061
:1032C000F0913503F1FD08C01091CF021F5F1093FC
:1032D000CF02F260F093350380E20E94BA0888239F
:1032E00079F0A0913503A2FD0BC040913C03411140
:1032F00001C041E0415040933C03A460A0933503DA
:1033000080E40E94BA08882371F0E0913503E3FD60
:103310000AC080913C03893008F48F5F80933C039E
:10332000E860E09335030E94B20887FD05C0009174
:1033300035030E70009335030E94B20884FD05C06A
:10334000209135032D70209335030E94B20885FD2E
:1033500005C0509135035B70509335030E94B2084D
:1033600086FD05C070913503777070933503909199
:103370002D039F5F903108F090E090932D0321E0A2
:1033800040E868E070E090E080E00E94C708F090BC
:10339000CF02E0903C0310921003109110031830FC
:1033A00008F0A3C2BBE01B9F4001112434019FEF32
:1033B000691A790A01E02AE04AE06AE070E0C30194
:1033C0000E94CF092AE04AE065E170E0C3010E9453
:1033D000CF09BE016F5F7F4F812F0E946B0CAC0144
:1033E0005980552079F083E0440F551F8A95E1F705
:1033F0004D57564F08E028E06BE070E0C40102969C
:103400000E943206BE016F5F7F4F88E0810F0E94ED
:103410006B0CAC01D980DD2079F003E0440F551F1F
:103420000A95E1F74D57564F08E028E066E170E055
:10343000C40102960E9432061F5F10931003ADCFA5
:1034400081FE09C031D9882309F473C133E0309378
:103450003E0310923D0340913D0342FF12C01430E1
:1034600080F01092CF0260913A0370913B0343FFCA
:1034700063C1477040933D03706870933B03609352
:103480003A0308E010E010932C0300932B0372E042
:10349000A72EB12CB0922A03A09229038CE798E0C2
:1034A0000E94740910932C0300932B038AE090E090
:1034B00090932A038093290387E798E00E94740978
:1034C00010932C0300932B03E2E1F0E0F0932A0326
:1034D000E093290381E798E00E947409AEE3B0E02D
:1034E000B0932C03A0932B03B0922A03A09229033C
:1034F00087E698E00E94740924E330E030932C03BF
:1035000020932B034BE050E050932A034093290370
:103510008AE598E00E94740980E10E94BA08882335
:1035200099F05091CF02543079F470913D0370932B
:103530002D031092CF02972F990F967009F491E006
:103540007870792B70933D0380E80E94BA08882335
:10355000A9F0B091CF02B43089F4F0913D03F0931B
:103560002D031092CF022F2F30E03595279527702D
:1035700009F424E0F870F22BF0933D03E0903D0352
:103580002E2D217044E064E070E081E090E00E9424
:10359000C7080E2D10E0980135952795217044E05D
:1035A0006CE070E081E090E00E94C70815950795F7
:1035B00015950795202F217044E064E170E081E0CB
:1035C00090E00E94C708E3FEBCC041E068E170E003
:1035D0008AE290E00E94050941E064E170E08AE23D
:1035E00090E00E94050941E066E170E08CE290E025
:1035F0000E94050941E066E170E088E290E00E94E7
:10360000050941E068E170E08BE290E00E94050965
:1036100041E068E170E089E290E00E94050941E044
:1036200064E170E08BE290E00E94050941E064E112
:1036300070E089E290E00E94050941E067E170E0F6
:103640008CE290E00E94050941E067E170E088E2C9
:1036500090E00E94050941E065E170E08CE290E0B5
:103660000E94050941E065E170E088E290E00E9477
:10367000050941E067E170E08CE290E00E940509F5
:1036800041E067E170E088E290E00E94050941E0D6
:1036900065E170E08CE290E00E94050941E065E19F
:1036A00070E088E290E00E94050941E068E170E086
:1036B0008BE290E00E94050941E068E170E089E258
:1036C00090E00E94050941E064E170E08BE290E047
:1036D0000E94050941E064E170E089E290E00E9407
:1036E000050980915C0290915D02892B09F472C0FA
:1036F00098E2492E512C10921003109110031031B2
:1037000008F0EBC06F2D812F0E94540AE8E08E9FD5
:10371000A0011124475B544F08E028E0B201A8E063
:103720001A9FC00111240E9432061F5F10931003DC
:10373000E4CF10923C038FCE486040933D037F77E7
:103740009CCE21E045E064E170E08AE290E00E94D6
:103750008E0921E045E064E170E08BE290E00E9498
:103760008E0921E043E065E170E08CE290E00E9488
:103770008E0921E045E064E170E089E290E00E947A
:103780008E0921E043E065E170E088E290E00E946C
:103790008E0921E043E065E170E08CE290E00E9458
:1037A0008E0921E045E064E170E08BE290E00E9448
:1037B0008E0921E043E065E170E088E290E00E943C
:1037C0008E0921E045E064E170E089E290E00E942A
:1037D0008E0987CF61E070E070935D0260935C02B8
:1037E00010921003E0911003E03208F081CFF0E076
:1037F000EE0FFF1FE053FD4F1182108210922D0338
:1038000000912D0310911003003108F062C01230B6
:1038100050F440E0612F802F0E943A0A40E0612F6F
:1038200081E0800F18C01230F1F40E94832890903C
:103830001003B0902D036AE070E00E94E12941E09E
:1038400005970CF440E0692D8B2D0E943A0A41E067
:10385000692D81E08B0D0E943A0A30912D033E5F65
:1038600030932D03CDCF133041F441E063E0802F3E
:103870000E943A0A41E063E0D3CF143041F442E0C1
:1038800064E0802F0E943A0A42E064E0C9CF15301C
:1038900021F70E9483286AE070E00E94E12942E05B
:1038A00005970CF043E06091100380912D030E9476
:1038B0003A0A0E9483286AE070E00E94E12942E00F
:1038C00005970CF043E080912D03609110038F5F0A
:1038D000C2CF1F5F1093100385CFF39448E0440ECE
:1038E000511C28E0F21207CFC0CC60913A036770F8
:1038F00009F4FEC008E028E04BEF59E06CE070E00E
:103900008EE590E00E94320640913A034770440FE2
:1039100021E06AE070E08DE590E00E94C7088091A8
:103920003A0390913B03B3E096958795BA95E1F7FA
:10393000877009F4E7C008E028E043E05AE06CE053
:1039400070E089E690E00E94320640913A0350917F
:103950003B03A3E056954795AA95E1F74770440FBE
:1039600021E06AE070E088E690E00E94C70880915C
:103970003A0390913B03F6E096958795FA95E1F727
:10398000877009F4C9C008E028E04BE05AE06CE019
:1039900070E085E790E00E94320640913A03509132
:1039A0003B03E6E056954795EA95E1F74770440FEB
:1039B00021E06AE070E084E790E00E94C70830915F
:1039C0003B033695377009F4B1C008E028E043E1C5
:1039D0005AE067E170E08EE590E00E943206409187
:1039E0003B034E7021E065E170E08DE590E00E94C0
:1039F000C70801E020E246E060E270E089E790E07D
:103A00000E94CF09F0913B03F295F77011E01F0F70
:103A100001E022E042E06CE370E08BE790E00E947E
:103A2000B20921E044E06BE370E08AE790E00E9495
:103A3000C708B12EBB0CBB0CB10E4BEF41036001AC
:103A40001124B601655C7F4F21E04B2D8BE790E0A0
:103A50000E948E09B601645C7F4F21E04B2D8CE7FC
:103A600090E00E948E0901E028E048E066E170E005
:103A700089E690E00E94B209A3E7B0E0B0932C037E
:103A8000A0932B03E7E1F0E0F0932A03E0932903EE
:103A9000809112030E94150F21E048E168E070E078
:103AA0008AE590E00E948E0981E08F1508F441C1FB
:103AB00070912D0397E09E1508F042C0793008F40C
:103AC000C8C092E1F99EB0011124675F7F4FEE2DCF
:103AD000E850FF0B9F01929FF001939FF00D11247E
:103AE00022E142E1CF01865A9F4F0E94CF09B1C027
:103AF00001E02AE04AE06AE070E08DE590E00E9493
:103B0000CF090DCF01E02AE04AE06AE070E089E6E3
:103B100090E00E94CF092BCF01E02AE04AE06AE062
:103B200070E085E790E00E94CF0949CF01E02AE0EC
:103B30004AE065E170E08DE590E00E94CF0959CF41
:103B4000793070F0BBE0FB9EB0011124675F7F4FBE
:103B500001E02CE04CE0EB9EC00111240E94CF0953
:103B6000BE016F5F7F4F8F2D880F880F880F8E0DDE
:103B70000E946B0C2C01898110922C0310922B0354
:103B800010922A0310922903882309F4CDC00E94C1
:103B9000150F68E070E070932C0360932B03109274
:103BA0002A031092290383E199E00E94740940E1FD
:103BB00050E050932C0340932B0310922A03109251
:103BC0002903FFE04F165104C0F4F201E651F24E12
:103BD0000C94F429F91D6A1E6D1E701E761E731E4C
:103BE000791E7C1E821E7F1E851E881E8B1E8E1EC9
:103BF000911E84E099E00E947409AEE6B0E0B093B3
:103C00002C03A0932B0310922A031092290380E126
:103C100099E00E94740910915E028EE099E01A30DA
:103C200030F08CE099E0143110F08AE099E00E94C5
:103C3000740988E00E94BA08882349F01F5F109336
:103C40005E021F3130F061E0C2010E94880D1092C7
:103C50005E0210921003A0905F02B0906002C090CC
:103C60006102D09062024FEFA416B406C104D104E1
:103C700009F09AC010925F021092600210926102E5
:103C80001092620200E0E0911003F0E0EB5EF64F6C
:103C900074903FEF731609F487C0AA24A394B12C43
:103CA000172D1770309010031A1508F456C0F5013F
:103CB000E30DF11DEB5EF64F84910E94790C6FEFDE
:103CC000A61AB60A8111ECCF130D1F5F10931003D3
:103CD0000F5FD9CF8BEF98E08ECF82EF98E08BCF3C
:103CE00087EE98E088CF82EE98E085CF87ED98E068
:103CF00082CF8CEC98E07FCF81EC98E07CCF84EB96
:103D000098E079CF87EA98E076CF81EA98E073CFA0
:103D100089E998E070CF8FE898E06DCF89E898E066
:103D20006ACF82E898E067CF82E899E00E94740940
:103D300090CF02E0F0128DCF27E02E1508F089CF4A
:103D400050912D03593008F484CF01E02AE044E279
:103D50006DE270E08AE590E0C8CEE12FE30DEF5F01
:103D6000E093100381E090E0A0E0B0E0002E04C0FA
:103D7000880F991FAA1FBB1F0A94D2F740915F02B8
:103D8000509160026091610270916202842B952BC8
:103D9000A62BB72B80935F0290936002A0936102E1
:103DA000B09362020F5F71CF01E020E247E760E26B
:103DB00070E081E090E00E94CF09F7E0FE1598F0F6
:103DC00081E08F1580F421E046E06CE270E082E053
:103DD00090E00E948E0921E043E06EE270E083E013
:103DE00090E00E948E0921E047E769E270E081E0FF
:103DF00090E00E94C70810921003E5E1F9E01491E9
:103E00005F2D22E0F21608F452E06EEF962E950E2A
:103E1000812C612C1F3F09F4D0C080915F029091EA
:103E20006002A0916102B0916202082C04C0B595B5
:103E3000A795979587950A94D2F780FF3DC080910A
:103E4000100396105AC12E2D4F2D60E00E94A70F2F
:103E500071E07F1580F597E09E1568F188E00E947B
:103E6000BA088823A1F050903203452D440F450D28
:103E700001E026E061E070E082E090E00E94B2099B
:103E8000B0913203B8322CF5BF5FB09332030E9479
:103E9000B20883FD10C01092320382E090E090934C
:103EA0002C0380932B0310922A03109229038CE396
:103EB00091E00E94070F6394E0911003EF5F177089
:103EC000E10FE0931003F0E0EB5EF64F1491839462
:103ED000A1CFB832E1F61092320362E070E0709345
:103EE0002C0360932B0310922A03109229038CE376
:103EF00091E00E94070FC0901003D12CF601EB5EF9
:103F0000F64F049110E053E0159507955A95E1F7A7
:103F1000B490F12CE12C4B2D4770E41690F4F6018F
:103F2000EA5EF64FEE0DFF1D8491682F677086954F
:103F30008695869590E00E94880D3FEFE31AF30A7C
:103F4000EACF0D31110508F027C0F801E655F04E13
:103F50000C94F429C71F322036203A203E204220FC
:103F600046204A204E2053205520572059205C20BF
:103F70005E20602062206520672069206B206E2013
:103F8000702072207420772079207B20462061E009
:103F900086E090E00E94C00D0FEF1FEF20E030E0C0
:103FA00000935F02109360022093610230936202DB
:103FB000A1E0A0933C031092CF0284E00E94BA08D3
:103FC000882329F031E0309333030E944211F091AD
:103FD0003E03F33009F0FDC7E0903D03E1106CC7EC
:103FE00080911303909114030E948628109212036B
:103FF0001092110321E02093330358E050932E03D5
:1040000010922F031092300310923203109231035A
:10401000109234031092350310923603109210035D
:10402000E0911003E03208F04AC6F0E0EE0FFF1F07
:10403000E053FD4F1182108210922D0300912D0349
:1040400010911003003108F036C6123008F0C3C5D5
:1040500040E0612F802F0E943A0A40E0612F81E00A
:10406000800FCFC561E089E090E094CF61E087E008
:1040700090E090CF61E088E090E08CCF61E08AE052
:1040800090E088CF61E08BE090E084CF61E08CE04D
:1040900090E080CF61E08EE090E07CCF61E080E056
:1040A0000E94050A79CF62E0FACF63E0F8CF64E0BE
:1040B000F6CF61E081E0F4CF62E0FCCF63E0FACFBD
:1040C00064E0F8CF61E082E0EBCF62E0FCCF63E038
:1040D000FACF64E0F8CF61E083E0E2CF62E0FCCFAA
:1040E00063E0FACF64E0F8CF61E084E0D9CF62E02A
:1040F000FCCF63E0FACF64E0F8CF292D30E02F5FEA
:104100003F4F6216130609F0D6CE2E2D4F2D61E0DB
:104110000E94A70FD0CE8091130390911403A09119
:104120001503B09116030196A11DB11D80931303D1
:1041300090931403A0931503B0931603D0FE03C00D
:104140000E94421120C0D1FE11C1809132038F5FC5
:1041500063E00E94C0299093320380E80E94BA086D
:1041600081110E94DA0A80E40E94BA08882309F4C7
:10417000CCC01092300384E00E94BA08882309F46E
:104180008AC00E94AA108EE293E00E94A90AA09120
:104190002F032A2F269526952695A03208F0DEC1FA
:1041A00010923C0341E04093CF024090CF0258E090
:1041B000541508F46BC21092100388E0489E7001F9
:1041C00011241091100390903C0300912F031031A3
:1041D00008F055C2692D812F0E94540A382EA12E55
:1041E000B12C3501B3E0660C771CBA95E1F778E0A5
:1041F000879FA0011124475B544F0770B701601BD4
:10420000710908E028E0C3010E94320695EF930D82
:10421000923008F0E2C1809127039091280368E76B
:1042200070E00E94CD29892B09F0D7C1292D30E0FB
:1042300080912F0386958695869590E0821B930B3F
:104240000596099708F0C9C180912E038695869539
:10425000869590E08A199B0907960F9708F0BDC1D3
:10426000B09111036B2F70E040E0A42E042E000CDF
:10427000BB08A616B7060CF078C1A6E0AA9DF0010F
:10428000AB9DF00D1124ED59FD4FD580DD2009F4D3
:1042900074C14F5FEACF10912E0360912F0370E03D
:1042A0006C5F7F4F43E0759567954A95E1F7212F45
:1042B00030E0C901049797FD079633E095958795FF
:1042C0003A95E1F70E94090B80932D03882311F0A2
:1042D000893091F41F5F10932E031770153060F032
:1042E000893051F410923D03F3E0F0933E03609166
:1042F00037036F5F6093370330912E033D3708F427
:1043000042CFECE7E0932E033ECF80E20E94BA0852
:10431000882321F1B1E0B093300384E00E94BA0811
:1043200081112FCF00912E0360912F0370E06C5FFD
:104330007F4F83E0759567958A95E1F7802F90E030
:10434000079623E0959587952A95E1F70E94240B1F
:10435000811119CF015000932E0315CF80903203A5
:10436000811011CF91E090933303EACED3FE18C0B1
:10437000809132038F5F63E00E94C02990933203E3
:10438000911105C071E0709333030E94421180E8DF
:104390000E94BA08882309F4F6CE0E94DA0AF3CE06
:1043A000D2FEF1CEB0913403B1113EC08AE00E943A
:1043B0008711882319F1BE016F5F7F4FCE010296EE
:1043C0000E943F0B882309F4DECE10923603E98168
:1043D000F0E0EE0FFF1FE053FD4FCA8021E030E018
:1043E00002C0220F331FCA94E2F740815181242B6F
:1043F000352B318320830E94B411C5CE70903603D3
:10440000772009F4C0CEF0903B03F7FEBCCE48E71E
:1044100040933F0350E45093900083E290E09093E8
:10442000990080939800AFCEB13009F03FC08AE088
:104430000E948711882309F4A6CE81E70E94790C97
:1044400011E0813009F010E089E60E94790C81309A
:10445000B1F432E0312BE0913803E13A08F530FF56
:1044600010C061E08EE090E00E94880D209138033A
:10447000213A08F020EA285D2093380384CE30E00A
:10448000E9CF327009F47FCE61E08DE090E00E94C8
:10449000880D209138032F3B08F02EEB265FECCFE0
:1044A000A32FA27089F730FF6ECEDBCFB230D1F4EC
:1044B0008AE00E948711882309F465CEF0E1F09329
:1044C0003303109235031092CF026FEF7FEF80E03D
:1044D00090E060935F02709360028093610290931A
:1044E000620251CEB33009F04ECE88E00E948711AF
:1044F000882309F448CE00911203002309F443CE27
:10450000BE016F5F7F4FCE0102960E94B20B809377
:104510002D03882309F437CE39806A8043E0632D68
:10452000862D0E943A0AE32DF0E0EE0FFF1FE053C4
:10453000FD4F81E090E002C0880F991F6A94E2F776
:10454000809590952081318182239323918380836C
:104550001092360301500093120315CE2350A03E53
:1045600008F028E120933C031DCEA616B70629F4D7
:10457000B13198F5BF5FB0931103413170F566E03A
:104580006A9DF0016B9DF00D1124ED59FD4F512FE7
:10459000550F550F550F5083FCE08FEF9FEF3F16DF
:1045A00011F081E090E006E00A9DF0010B9DF00D16
:1045B0001124ED59FD4F281B390B220F220F220F1A
:1045C0002183128263E06383309137033695365F2F
:1045D0003583892DC9D69F5F9483B0903403B11081
:1045E0001DC0BE016F5F7F4FCE0102960E943F0B40
:1045F00080932D03882391F0CA801C110FC08980FD
:1046000098100CC020912F032770B701621B71090D
:1046100000E028E048E0C3010E94CF097091340314
:10462000733049F530901203332029F1BE016F5FDA
:104630007F4FCE0102960E94B20B80932D038823F8
:10464000D1F09A81191317C0B9819B1214C00E942E
:10465000240760FD10C040912F034770B701641B11
:1046600071096F5F7F4F06E026E049E85BE0C30118
:1046700001960E9432061F5F10931003A2CD9394FF
:1046800090923C0343944092CF028FCD10912F0320
:10469000A0E43A2E310E103E30F4312EA0E2A117E4
:1046A00010F4F0E23F2E412C80912F037090110303
:1046B000471408F0E6C1A42CB12C66E06A9DA00165
:1046C0006B9D500D11248A010D591D4F6801F80191
:1046D000F580FF2009F450C1E32CE81A01810E0D8A
:1046E00001340CF049C17601C6010E94A90A9090DC
:1046F000270390FC2CC0D6011C9160902E03812FC3
:104700008619212F30E018160CF063C171E0F60114
:1047100072836180712C4901F7E08F0E911C73E068
:10472000959487947A95E1F7B3016C5F7F4FE3E04E
:1047300075956795EA95E1F7882D0E94240B811104
:104740001DC11150D6011C93C7010E94250A66E0C5
:104750006A9DF0016B9DF00D1124ED59FD4F4481D0
:10476000142F13708FEF810F8093CF0250E0559577
:10477000479555954795437055274150510923E07A
:10478000440F551F2A95E1F738E1839F400D511DD5
:104790001124F281F13009F071C184E090E0480FFA
:1047A000591F455E554F602F000F770B06E00A9D9D
:1047B000D0010B9DB00D1124AD59BD4F8C9190E0EF
:1047C00008E024E002960E9432062091370364E05C
:1047D0002A3038F063E0243120F062E0283208F01B
:1047E00061E070E08091270390912803D6D5892B52
:1047F00009F0B3C086E08A9DF0018B9DF00D112475
:10480000ED59FD4F818190912F03891B082E000CDB
:10481000990B97FF03C091958195910905970CF02D
:10482000ABC046E04A9DF0014B9DF00D1124ED59BF
:10483000FD4F0081A0902E0352E0D52EDA1874E0CF
:104840002A3038F078E0243120F07CE0283208F07B
:1048500070E1179FB02C112456D410913A031770B1
:1048600064E670E0AED52AE0129F4001112488155D
:10487000990524F493E0199FB018112444D4209191
:104880003A0330913B03B3E036952795BA95E1F7AB
:10489000277064E670E095D5BFE02B9F700111246E
:1048A0008E159F0524F463E0269FB01811242BD4A5
:1048B00020913A0330913B03A6E036952795AA95BF
:1048C000E1F7277064E670E07CD534E1239F300186
:1048D00011248615970524F483E0289FB01811242D
:1048E00012D470903B03172D1695177064E670E094
:1048F00068D5FEE11F9FD00111248A179B0724F47D
:1049000043E0149FB01811240D0D053030F51B1431
:1049100024F58091380390E08B199109B7FC9395A9
:1049200097FD80E08093380377FE0CC0E4E1E093CC
:104930003F0300E40093900024E335E030939900B6
:104940002093980053E254BD7FEF78BD91EF909390
:1049500080001092880070938A00C0902703C0FCEA
:104960000BC0B3E2B4BD6FEF68BD31EF3093800090
:104970001092880010928A00439496CE6301F4E06E
:10498000CF1AD108D7FE04C0630123E0C20ED11CA8
:1049900063E0D594C7946A95E1F76C2D882D0E9449
:1049A000240B8111D4CE6C2D812F8695869586950A
:1049B0000E94540A8111CBCE96E09A9DF0019B9DF6
:1049C000F00D1124ED59FD4F11501083B8E0B38361
:1049D000BBCE882309F4BBCEF60112826180712C14
:1049E0004901F3E08F1A910897FE04C0490144E0A1
:1049F000840E911C43E0959487944A95E1F7B301A6
:104A00006C5F7F4F53E0759567955A95E1F7882D58
:104A10000E94090B81110AC026E02A9DD0012B9D1E
:104A2000B00D1124AD59BD4F1F5F8DCE630154E011
:104A3000C51AD108D7FE04C0630163E0C60ED11CBD
:104A400033E0D594C7943A95E1F76C2D882D0E94F8
:104A5000090B81117CCE6C2D812F869586958695CC
:104A60000E94540A811173CE36E03A9DF0013B9DBD
:104A7000F00D1124ED59FD4F1F5FA7CF90E080E0AE
:104A80008ECE40903303442D50E09A013595279502
:104A9000242910E020FD15C0142D187043FC10C00F
:104AA00042FE0CC0F0913403FF2309F480C0F130C2
:104AB00009F47FC0F23029F0F33019F0122D01C053
:104AC00016E0A0913203A10FA09310031092CF0221
:104AD00040913003413031F4A45FA0931003E4E02F
:104AE000E093CF02803E08F466C0805C80932D0383
:104AF0002090100308E0209EA00111244D59554F2D
:104B000060912D0370E080912E039091CF0208E018
:104B100028E0891B990B0E94320600E028E048E05B
:104B200061E070E088E790E00E94B20930903403C1
:104B300028E0329EA0011124475D544F08E028E090
:104B400061E070E088E790E00E9432065091350302
:104B5000552319F051505093350300E028E047E405
:104B600061E070E081E390E00E94B209E2E3FE2E92
:104B700090903803892D6AE0F7D3581608F5752D03
:104B80007170A72E43E25BE050FE02C046E25BE09C
:104B900008E023E061E070E08F2D90E00E94320693
:104BA00094E0A11001C093E0F90E5394E1CF13E01B
:104BB00088CF19E086CF803208F498CF80E296CF74
:104BC000911003C0B4E0B0933E0310923C031092E6
:104BD000CF02212EFCC91230E1F495D2D0901003FF
:104BE000C0902D036AE070E0ECD341E005970CF42F
:104BF00040E06D2D8C2D0E943A0A41E06D2D81E040
:104C00008C0D0E943A0A70912D037E5F70932D03E4
:104C100015CA133041F441E063E0802F0E943A0A44
:104C200041E063E01CCA143041F442E064E0802FAC
:104C30000E943A0A42E064E012CA1530E1F463D2FD
:104C40006AE070E0BED342E005970CF043E060916B
:104C5000100380912D030E943A0A55D26AE070E059
:104C6000B0D342E005970CF043E080912D036091B2
:104C700010038F5FC6CFFF24F394F00E1E3149F46A
:104C800040E06EE1802F0E943A0A40E06EE18F2DF5
:104C9000B8CF1F3141F448E06FE1802F0E943A0AFB
:104CA00048E06FE1F4CF43E0612F802F0E943A0A81
:104CB00043E0612FECCF1F5F10931003B1C923D2E3
:104CC00064E070E07ED3809310031DD22C011BD2D0
:104CD0005C0119D24C01C2016AE070E072D342E07B
:104CE000480FC50164E170E06CD3E8E0E80FC4014F
:104CF0006CE070E066D36E2F8E5F0E94BF129091C1
:104D000010039F5F909310039830F8F2FCD164E099
:104D100070E057D380931003F6D1709037037694E8
:104D200064E670E04ED3870D8093CF0204E08832B2
:104D300050F005E0863438F007E08F3520F00AE0C7
:104D4000833708F006E0DFD13C01DDD17C01DBD107
:104D50006C01C30162E070E034D341E0480FC70149
:104D600069E170E02ED336E0380FC6016CE070E0E8
:104D700028D3202F632F8E5F0E947E12B0911003E4
:104D8000BF5FB0931003B83108F4C6CFBCD164E65E
:104D900070E017D3C2970CF06FC0B5D166E170E038
:104DA00010D3382E56E0552E580EADD16BE070E082
:104DB00008D3182F482E63E0A62EA80EFB80842C63
:104DC0008F0C40E0652D882D0E943A0A97E0792EDD
:104DD000730C40E0672D882D0E943A0A28E0922E3D
:104DE000930C40E0692D882D0E943A0A35E0B32EDD
:104DF000B30C64E0630D6F0D48E081E0840D0E9408
:104E00003A0A48E06B2D882D0E943A0A49E0D42ED8
:104E1000D30C48E06D2D882D0E943A0AF39466E089
:104E2000F612CDCF1B5F48E06B2D812F0E943A0A0E
:104E300048E0652D812F0E943A0A48E0672D812FB6
:104E40000E943A0A48E0692D812F0E943A0A48E000
:104E50006D2D812F0E943A0A4BE0692D8A2D0E9408
:104E60003A0A47E0AEEF4A1508F4A2E040E0692DA7
:104E7000AA1A8A2D0E943A0A80913703F82FF770F8
:104E800049F4882339F03FD160E170E09AD2885F1D
:104E90000E94F80D48E06DE18EE00E943A0A48E079
:104EA0006DE18FE00E943A0A49E06EE18FE00E94D6
:104EB0003A0A21E020933D0350913C035F5F752F38
:104EC000593008F078E070933C03583018F188E0CE
:104ED0000E94BA08882381F0E3E2E4BD9FEF98BD09
:104EE00001EF009380001092880010928A0032E057
:104EF00030933E0310923D0384E00E94BA08882359
:104F000009F4B7C0B0913203BF5FB9320CF065C08D
:104F1000B0933203809127039091280387709927DB
:104F2000892B59F443E244BDFFEFF8BD21EF2093F4
:104F300080001092880010928A0010922C03109228
:104F40002B0310922A0310922903E0903703E0927A
:104F50002D0389EE9BE00E947409E4E2F0E0F093F7
:104F60002C03E0932B0310922A03109229038E2D19
:104F70000E94150F10922C0310922B0300E110E0F9
:104F800010932A030093290388ED9BE00E94740983
:104F900010922C0310922B03A0E2B0E0B0932A03EE
:104FA000A093290389EC9BE00E94740901E024E0AE
:104FB00040E56AE270E090E080E00E94CF09409115
:104FC0003203440F22E06BE270E090E080E00E9448
:104FD000B2090E94C4080C94AC18109232036EEB14
:104FE0008FEF90E00E94AE1369E780E091E00E94AD
:104FF000AE1361E081E091E00E94AE13609137034F
:1050000082E091E00E94AE136091380383E091E06A
:105010000E94AE1360913B0384E091E00E94AE13C6
:1050200060913A0385E091E00E94AE1360913903EC
:1050300086E091E00E94AE1387E1682E83E0782E2F
:1050400007E011E0D3016D913D01C8010E94AE134C
:105050000F5F1F4F0731F1E01F07A1F713E214BDE7
:1050600018BC61EF609380001092880010928A0053
:1050700051CF109232034ECF8F929F92AF92BF9238
:10508000CF92DF92EF92FF92CF93DF93EC01688192
:1050900079818A819B81611571058105910521F4D2
:1050A00064E279ED8BE597E02DE133EF41E050E0EC
:1050B000FED049015A019B01AC01A7EAB1E413D12A
:1050C0006B017C01ACEEB4EFA501940118D1DC01B9
:1050D000CB018C0D9D1DAE1DBF1DB7FF03C00197F9
:1050E000A109B04888839983AA83BB839F77DF9106
:1050F000CF91FF90EF90DF90CF90BF90AF909F90B7
:105100008F900895B9CF8DE091E0B6CFB0E0A0E0E8
:1051100080930D0190930E01A0930F01B0931001A5
:1051200008958F929F92AF92BF92CF92DF92EF92AB
:10513000FF92CF93DF93EC01688179818A819B8113
:10514000611571058105910521F464E279ED8BE526
:1051500097E02DE133EF41E050E0A9D049015A0139
:105160009B01AC01A7EAB1E4BED06B017C01ACEEBF
:10517000B4EFA5019401C3D0C60ED71EE81EF91ED8
:10518000F7FE06C081E0C81AD108E10880E8F80AF5
:10519000C882D982EA82FB82C701B6019F77DF917C
:1051A000CF91FF90EF90DF90CF90BF90AF909F9006
:1051B0008F9008958F929F92AF92BF92CF92DF927D
:1051C000EF92FF9260911101709112018091130191
:1051D00090911401611571058105910521F464E236
:1051E00079ED8BE597E02DE133EF41E050E05FD0C2
:1051F00049015A019B01AC01A7EAB1E474D06B01EB
:105200007C01ACEEB4EFA501940179D0C60ED71E97
:10521000E81EF91EF7FE06C081E0C81AD108E108B1
:1052200080E8F80AC0921101D0921201E0921301B5
:10523000F0921401C701B6019F77FF90EF90DF90C5
:10524000CF90BF90AF909F908F9008956093110181
:105250007093120180931301909314010895F999AA
:10526000FECF92BD81BDF89A992780B50895262F6B
:10527000F999FECF92BD81BDF89A019700B402164C
:1052800039F01FBA20BD0FB6F894FA9AF99A0FBEFA
:105290000895262FF999FECF1FBA92BD81BD20BD7A
:1052A0000FB6F894FA9AF99A0FBE01960895052E52
:1052B00097FB16F400940FD057FD05D024D007FCBF
:1052C00002D046F408C050954095309521953F4F47
:1052D0004F4F5F4F089590958095709561957F4FE2
:1052E0008F4F9F4F089531D0A59F900DB49F900D83
:1052F000A49F800D911D11240895B7FFF4CFF3DF13
:10530000821B930B0895A1E21A2EAA1BBB1BFD0161
:105310000DC0AA1FBB1FEE1FFF1FA217B307E40794
:10532000F50720F0A21BB30BE40BF50B661F771FEC
:10533000881F991F1A9469F76095709580959095CC
:105340009B01AC01BD01CF010895A29FB001B39FA5
:10535000C001A39F700D811D1124911DB29F700D7E
:10536000811D1124911D0895991B79E004C0991F96
:10537000961708F0961B881F7A95C9F780950895AF
:1053800087FB082E062687FD819567FD6195ECDF7A
:105390000EF4919507FC81950895AA1BBB1B51E162
:1053A00007C0AA1FBB1FA617B70710F0A61BB70B95
:1053B000881F991F5A95A9F780959095BC01CD013A
:1053C000089597FB072E16F4009406D077FD08D0B9
:1053D000E4DF07FC05D03EF4909581959F4F08953A
:1053E000709561957F4F0895EE0FFF1F0590F49122
:1053F000E02D09942F923F924F925F926F927F928D
:105400008F929F92AF92BF92CF92DF92EF92FF92D4
:105410000F931F93CF93DF93CDB7DEB7CA1BDB0B80
:105420000FB6F894DEBF0FBECDBF09942A88398825
:1054300048885F846E847D848C849B84AA84B9842C
:10544000C884DF80EE80FD800C811B81AA81B98138
:10545000CE0FD11D0FB6F894DEBF0FBECDBFED014C
:065460000895F894FFCF4F
:10546600FFFFFFFF00E10000000000001001000048
:10547600000100000000C180810000000000000063
:105486005508E60777086C0895087A08860800002C
:1054960000002009C307BB0EBA0E7800486F6C6483
:0C54A600204120546F20437261667400A6
:00000001FF
